:100000000C9426040C9443040C9443040C94430471
:100010000C9443040C9443040C9443040C94430444
:100020000C9443040C9443040C9443040C94430434
:100030000C9443040C9443040C9443040C94430424
:100040000C94F2070C9461050C9443040C94430443
:100050000C9443040C9443040C9443040C94430404
:100060000C9443040C9443040C9443040C944304F4
:100070000C9443040C9443040C9443040C944304E4
:100080000C9443040C9443040C944304071EEC1F8B
:100090000C1ED71F231E231E5D1E721EA41EF31EE0
:1000A0006F1EEC1FEC1F881F9A1FB81FC61FEC1F86
:1000B000EC1FEC1FEC1FEC1FEC1FEC1FEC1FEC1FE8
:1000C000EC1FEC1FEC1FDB1FDD1FE21F4561737986
:1000D000436F6E74726F6C00204C4300696E636FE7
:1000E0006D70617469626C6520485700312E342E42
:1000F00032000102031304050611070809120A0061
:100100000B0C100F0E0D010101050D1F0C04040E48
:100110001F04041F0E040006091717090600000635
:1001200009121412090603070F1E1C1810000305FC
:100130000912141810000707070707070707070524
:100140000505050505071C101817150705071C10E0
:100150001817110202021C101812140605021C10B6
:100160001817140601061C101815150701011C109C
:100170001816110201061C101816110204071C1093
:10018000181216020207040A110A0A0E00000C17C0
:10019000141714170C001C101810160505051F0A5B
:1001A0000A0A0A0A1F000E11111F1B1B1F0002065C
:1001B0000F1F0F060200080C1E1F1E0C08000E0E5B
:1001C0000E0E1F0E0400040E1F0E0E0E0E00202039
:1001D000202020200000204D4D4920200000204DEF
:1001E0004D012020000020444343202000002053E4
:1001F000544F5020000053484F52542100002048D3
:10020000414C54200000000000000000000020507D
:10021000524F4720000052455345542000007E0EA7
:100220000E0E0E1B1B1C0E1B1B7E0E0E0E0E232D08
:10023000004144523A20256C6420202020202020B8
:10024000202020002D2D2D2D202000252D3564006F
:1002500025336400202001022020202020202000BF
:10026000252D356400252D31312E31317300414269
:10027000434445464748494A4B4C4D4E4F505152D6
:10028000535455565758595A30313233343536371E
:1002900038392E2C3A2D2B232F3D3C7C3E20004D0F
:1002A0004D20492020313420004D4D20492020325E
:1002B0003761004D4D20492020323762004D4D20DE
:1002C000012020313420004D4D20012020323761A3
:1002D000004D4D200120203237620044434320204E
:1002E0002031342000444343202020323820004471
:1002F0004343202031323820004C6F636D656E75AA
:1003000000000000000000000044434320686F6FBD
:10031000666473706F6F7200004C434420766572A0
:100320006C69636874696E67004C6F6B436F6E74C1
:10033000726F6C00000000000045786974000000D6
:100340000000000000000000004B69657A656E2027
:1003500000000000000000000044617461666F72DC
:100360006D61740000000000004E61616D2020206E
:10037000202020000000000000496E766F6572208A
:100380002020200000000000004D656E75204C6F9D
:10039000636F0000000000000050726F6772616DB3
:1003A0006D6174696F6E0000004C756D696E6F73DE
:1003B0006974650000000000004C6F6B436F6E7441
:1003C000726F6C0000000000004578697400000046
:1003D00000000000000000000053656C6563746954
:1003E0006F6E20000000000000466F726D61742087
:1003F000646F6E6E65657300004E6F6D2020202067
:10040000202020000000000000536169736965200E
:100410002020200000000000004C6F6B204D656E16
:10042000FC000000000000000044434320486175C8
:100430007074676C65697300004C43442042656CBE
:100440006575636874756E67004C6F6B436F6E748F
:10045000726F6C00000000000045786974000000B5
:1004600000000000000000000041757377E4686C34
:10047000656E20000000000000446174656E666FC8
:10048000726D617400000000004E616D65202020D7
:1004900020202000000000000045696E7472616732
:1004A0002020200000000000004C6F636F6D6F740F
:1004B000697665206D656E7500444343204D616922
:1004C0006E20547261636B00004C43442062616390
:1004D0006B6C696768740000004C6F6B436F6E74DF
:1004E000726F6C0000000000004578697400000025
:1004F00000000000000000000053656C656374207C
:100500000000000000000000004461746120666F7C
:10051000726D617400000000004E616D6520202046
:10052000202020000000000000456E747279202019
:10053000202020000000000000202D2D2D2D002562
:10054000357500536F6674772E205600312E342E89
:1005500032005365724E722E2025386C75003A2099
:100560000025357500253364002534643A20002DBC
:100570002D2D0025336400204F4B2020202000200B
:1005800020202020202000696E636F6D7061742E22
:1005900020466F726D617400496E636F6D702E201E
:1005A000466F726D6174202000466F726D61742019
:1005B000696E636F6D7061742E00696E6B6F6D7024
:1005C00061742E20466F726D6174002E2E2E20777E
:1005D000616974696E67202E2E2E2000233D6465AC
:1005E0006C657465000000000000000000286E6F5C
:1005F00020656E74727929000000000000002E2E24
:100600002E2064656C6574696E67202E2E2E002086
:100610006661756C740000000000000000000000BE
:1006200020444343206F6E6C7921000000000000DD
:10063000002A3D43616E63656C20202000000000AD
:1006400000002070726F6772616D696E6700000054
:100650000000002D73686F7274206369726375699E
:10066000742D20002E2E2E207761636874656E2015
:100670002E2E2E2000233D77697373656E000000D7
:10068000000000000000286765656E20696E766FC7
:1006900065722900000000202E2E2E2077697373CA
:1006A000656E202E2E2E000020666F7574000000EF
:1006B00000000000000000000020416C6C65656EC9
:1006C000204443432100000000002A3D204166628F
:1006D00072656B656E0000000000002050726F674D
:1006E00072616D6D6572656E000000002D2D4B6F9F
:1006F0007274736C756974696E672D2D0050617426
:1007000069656E74657A0000000000000000233DFA
:100710007375707072696D6572000000000000767C
:100720006964650000000000000000000000000097
:100730005375707072657373696F6E00000000000E
:100740000020457272657572000000000000000014
:1007500000002044434320756E697175656D656EB8
:100760007400002A3D4162616E646F6E20200000BB
:10077000000000002050726F6772616D6D617469D6
:100780006F6E0000002D436F7572742D6369726384
:100790007569742D20002E2E2E2077617274656E7F
:1007A000202E2E2E202000233D4CF6736368656EAC
:1007B0000000000000000000286B65696E2045699C
:1007C0006E7472616729000000202E2E2E206CF6B8
:1007D00073636865202E2E2E2000204665686C65A8
:1007E0007200000000000000000000206E75722002
:1007F00066FC722044434321000000002A203D2073
:10080000416262727563680000000000002050724F
:100810006F6772616D6D696572756E6700002D2D71
:10082000204B75727A7363686C75DF202D2D005B29
:100830006E6F206D6573736167655D005B756E6BD0
:100840006E6F776E206572726F725D0011241FBE2D
:10085000CFEFD0E1DEBFCDBF11E0A0E0B1E0E6E92F
:10086000FBE400E00BBF02C007900D92A033B1077C
:10087000D9F713E0A0E3B1E001C01D92A834B1079D
:10088000E1F70C947D040C94000081E08093310129
:100890000895482F90913001981731F0963021F04B
:1008A000953029F4863019F080E090E00895409367
:1008B0003001453021F460E280E00E942F20409119
:1008C0003001463021F460E280E00E942F200E9437
:1008D000450481E090E008950895809130019927C2
:1008E00008950E94D11D0E94EF0F8091310188234D
:1008F00011F40E94480BA8950895CFEFD0E1DEBF18
:10090000CDBF0E944E1B0E941D050E944205789497
:100910000E94A2070E94741BFC0184810E94B10BFB
:100920006CEC70E082E00E94D40B0E948A1B823043
:1009300079F00E948A1B813059F060E081E00E94CA
:100940005E0A6CED70E082E00E94D40BA895FECFA9
:1009500068ED70E082E00E94D40B60E081E00E94CC
:100960005E0A66E582E00E94B60B6CEE70E082E003
:100970000E94D40B0E94741B8C0181E00E945909D3
:10098000882319F081E00E94771B82E00E945909B8
:10099000882319F080E00E94771B83E00E945909A8
:1009A000882319F082E00E94771B84E00E94590995
:1009B000882329F083E00E94771B01C0A8950E943C
:1009C000F01C8823D9F3F80181859285892BC9F021
:1009D0000E94680CEC0144969E01215F3F4FAC01E0
:1009E000B901F801818592850E943521BC01892BCE
:1009F00029F0F801818592858A8B9B8B61157105A1
:100A000019F4F801628173818FEF0E94EB1B81E082
:100A100011C00E940A100E940A0AFFEF8F3F9F0731
:100A2000C1F70E947104809131018823A1F31092D3
:100A3000310180E00E94F50DEECF8FE78ABB1BBA33
:100A400080E187BB18BA80EF84BB8FEF85BB8BEB4F
:100A500081BB8CEC82BB86E082B987EF83B980933F
:100A6000610081EF809362008FE18093640089E1EF
:100A7000809365000E94D308A89588E181BD8CE031
:100A800081BD08950E947C1B9B01AC0193E0E92F7E
:100A9000FF27E45CFE4F822F8F77808387E0569597
:100AA0004795379527958A95D1F7915097FFEFCFC6
:100AB00087B3807F87BB88B3807F88BB84EE8DB986
:100AC00008951F920F920FB60F9211242F933F9308
:100AD0004F935F936F937F938F939F93EF93FF93C6
:100AE00080910001909101018F5F9F4F71F0BB9A3F
:100AF000809100018FB9769B0BC0BB981092320198
:100B0000109239011092380103C0BB988FEF8FB952
:100B10007FB177FF7FC080913A0190913B01892B93
:100B2000E1F0809136018F5F80933601809136012C
:100B3000803210F010923601909136018091370189
:100B4000981759F4809137018F5F80933701809116
:100B50003701803210F01092370180913801909166
:100B600039018D5D924061F058F0809135018F5FC1
:100B70008093350180913501843010F01092350159
:100B800010923B0110923A011092390110923801F3
:100B900060912F01761721F481E08093320171C0BA
:100BA00010923201472F55279A012F773070862FE8
:100BB00099272817390721F07F3F11F06F3F61F423
:100BC0009091360189E0989FC001112483549E4F73
:100BD00090933B0180933A014F775070862F99276D
:100BE0004817590709F04DC09091340180913501A3
:100BF000981749F09091350189E0989FC001112420
:100C000083529D4F02C084EB91E090933901809311
:100C1000380137C020913201822F99278130910508
:100C200031F0813091056CF106975CF516C02F5FAD
:100C300020933201703419F41092330122C07134C0
:100C400011F481E007C0723411F482E003C0733400
:100C500091F483E08093330114C0E22FFF27809149
:100C60003301992702968E179F0744F0E65CFE4FEA
:100C70008081781719F01092320103C02F5F209302
:100C8000320180913201882339F4809138019091AA
:100C90003901892B79F003C0872F99270DC0E09186
:100CA0003801F091390181919927F0933901E0934E
:100CB000380102C08FEF9FEF9093010180930001F4
:100CC00080913A0190913B018D5D924020F010920D
:100CD0003B0110923A01E0913A01F0913B013097CB
:100CE00029F07193F0933B01E0933A01FF91EF916A
:100CF0009F918F917F916F915F914F913F912F9134
:100D00000F900FBE0F901F901895DC018091340159
:100D1000282F332780913501992701972817390704
:100D200041F080913401833039F48091350188237A
:100D300019F480E090E008959091340189E0989F43
:100D4000F0011124E352FD4F98E08D918193915071
:100D500097FFFBCF809134018F5F809334018091A6
:100D60003401843010F01092340181E090E0089555
:100D70000895FC01A4EBB1E098E081918D9391502E
:100D800097FFFBCF08959C01909136018091370128
:100D9000981719F480E090E00895D90121153105E4
:100DA00011F4C9010895F8949091370189E0989F52
:100DB000F0011124E354FE4F98E081918D939150FE
:100DC00097FFFBCF809137018F5F80933701809130
:100DD0003701803210F0109237017894C9010895DC
:100DE000089500000000000000000895882341F0ED
:100DF000809165008460809365000E94F1060895EB
:100E0000809165008B7F80936500089508959B0114
:100E1000AC018091030390910403A0910503B0916C
:100E2000060382179307A407B507A0F08091030378
:100E300090910403A0910503B0910603821B930BCC
:100E4000A40BB50B80509041A040B040A0F080E0D2
:100E500090E008958091030390910403A09105030D
:100E6000B0910603281B390B4A0B5B0B2050304F07
:100E70004F4F5F4F18F081E090E0089580E090E0E0
:100E800008950895EF92FF920F931F93AA27BB270F
:100E9000E0900303F0900403009105031091060312
:100EA000E80EF91E0A1F1B1F01C0A895C801B70153
:100EB0000E9407078823C9F31F910F91FF90EF90BD
:100EC00008950F931F93CF93C82F162F042F80914F
:100ED00065008D7F8093650080E00E94F6068AB3EE
:100EE0008F608ABB8BB3807F9C2F92959F70892BDC
:100EF0008BBB112321F080916500816003C080913C
:100F000065008E7F8093650081E00E94F60680E098
:100F10000E94F606002329F088E090E00E94420734
:100F20000DC08BB3807FCF708C2B8BBB0E94F106E2
:100F300081E00E94F606802F0E94F606CF911F9155
:100F40000F91089588E290E00E94420741E060E03E
:100F500080E30E94610741E060E080E30E94610756
:100F600041E060E080E30E94610741E060E080E2F0
:100F70000E94610788E20E94540A88E00E94540A95
:100F800081E00E94540A86E00E94540A8CE00E948C
:100F9000540A66EC71E080E00E948D0B6EE971E00E
:100FA00081E00E948D0B66EA71E082E00E948D0B69
:100FB0006EE871E083E00E948D0B6EE771E084E0E3
:100FC0000E948D0B66E771E085E00E948D0B6EE656
:100FD00071E086E00E948D0B66E671E087E00E947A
:100FE0008D0B08951F920F920FB60F9211241F932D
:100FF0002F933F934F935F936F937F938F939F9321
:10100000AF93BF93EF93FF9380914201882309F040
:10101000B8C081E0809342017894809140018F5F55
:1010200080934001282F237009F0A9C086958695EA
:101030008770992783309105C1F1843091052CF494
:10104000009759F00197E9F09AC08530910509F4AD
:1010500060C0079709F491C092C0809103039091FA
:101060000403A0910503B09106030196A11DB11DD3
:101070008093030390930403A0930503B0930603A6
:101080007EC08091030390910403A0910503B09169
:10109000060381709070A070B070892B19F00E94C7
:1010A0006C096DC00E942D096AC08091410188239E
:1010B00009F465C08AB3807F8ABB822F0E94F6063E
:1010C00080916500826080936500809165008E7FCD
:1010D000809365000000000081E00E94F60619B3CD
:1010E00080E00E94F6061295107F0E94F10681E0D2
:1010F0000E94F60689B38F70182B80E00E94F606D6
:10110000812F992787FD90958827990F881F992708
:1011100031C060914101662391F590910703809160
:101120000803981789F010910803E12FFF27E95F62
:10113000FC4F82811F5F103108F0162F803891F428
:1011400080910703811719F480E090E013C0E12F2C
:10115000FF27E95FFC4F82811F5F103108F0162FD7
:10116000462F02C0462F61E00E94610710930803DA
:1011700081E090E08093410102C00E94F00910924A
:101180004201FF91EF91BF91AF919F918F917F911C
:101190006F915F914F913F912F911F910F900FBED3
:1011A0000F901F90189510927D0017BE11BE89E612
:1011B00083BF87B7816087BF0895EF92FF920F9337
:1011C0001F93AA27BB27E0900303F090040300912C
:1011D000050310910603E80EF91E0A1F1B1F02C02B
:1011E0000E947104C801B7010E9407078823C1F358
:1011F0001F910F91FF90EF900895282F220F6111FA
:101200002160822F83708150823028F424FF02C035
:101210002E6001C0217F822F99270895909145016A
:10122000E92FFF27EB5BFE4F8283892F8F5F80932F
:101230004501883010F0109245019091460180914F
:101240004501981741F4892F8F5F809346018830BC
:1012500010F010924601089508950F931F9311B155
:10126000812F8074682F809143010E94FD08082F10
:10127000809343011078612F809144010E94FD0802
:1012800080934401007C807C003829F4882339F065
:10129000803C61F408C0003449F4803C11F484E1DE
:1012A00003C0882319F485E10E940E091F910F9154
:1012B0000895843118F080E090E0089520E030E057
:1012C000E82FFF27E15BFE4F8081882311F021E0AA
:1012D00030E0C90108950895FF920F931F93CF93B3
:1012E00080916801E82FFF27ED59FE4F008113B36D
:1012F0001083FF2480916801E82FFF27EE0FFF1F66
:10130000EE0FFF1FEF0DF11DEE50FF4FC49110FDCA
:1013100031C000FF14C0C23129F481E10E94590993
:10132000882331F48C2F0E940E09C43108F043C089
:10133000EC2FFF27E15BFE4F81E080833CC0C4318E
:10134000D0F5EC2FFF27DF01A15BBE4F9C919F5F83
:101350009C93992311F49F5F9C937197329758F552
:1013600080916001893738F180916101893718F1E6
:1013700085E01FC0C43128F4EC2FFF27E15BFE4F4E
:10138000108200FD18C08C2F80680E940E090E94F8
:101390006D04853081F4C13121F482E10E94590944
:1013A00005C0C23141F481E10E945909882319F432
:1013B00086E00E94490416950695F39483E08F1504
:1013C00008F098CF809168018F5F80936801853025
:1013D00010F010926801CF911F910F91FF90089526
:1013E00090916801943029F485B3806F85BB9798FC
:1013F0000895979A85B38F7020E130E002C0220FE4
:10140000331F9A95E2F7922F9095907F892B85BB99
:10141000089508958091450120914601821719F49D
:101420008FEF9FEF0895E22FFF27EB5BFE4F828146
:10143000482F5527822F8F5F80934601883010F008
:1014400010924601CA0108950895CF93C82F07C08E
:1014500080910803882391F40E94D11DA895809162
:101460000703282F3327809108039927019728170E
:10147000390791F3809107038F3051F3F8948091ED
:101480000703E82FFF27E95FFC4FC2838091070322
:101490008F5F8093070380910703803110F01092D3
:1014A00007037894CF9108951F93182F80E80E9426
:1014B000250A812F0E94250A1F9108958295880F81
:1014C000880F807C860F80680E94540A08950E94CD
:1014D0005E0A8EE00E94540A08958CE00E94540A2D
:1014E0000895FF920F931F93CF93F82E60912A03D4
:1014F000809129030E945E0AC0E009E113E0809117
:101500002B03C81778F4FF2021F0F80161918F01B7
:1015100001C060E282E00E94B60BCF5F80912B0396
:10152000C81788F3CF911F910F91FF900895909362
:10153000340380933303892B89F1709332036093D2
:101540003103CB01AA27BB27209103033091040369
:101550004091050350910603280F391F4A1F5B1F56
:1015600020932D0330932E0340932F035093300389
:1015700080912C038E7F80932C032115310541052A
:10158000510561F42F5F3F4F4F4F5F4F20932D0365
:1015900030932E0340932F03509330030895089502
:1015A000AF92BF92CF92DF92EF92FF920F931F9371
:1015B000CF93DF93D82EC62EEA0189E1E82E83E08F
:1015C000F82E109234031092330381E08D1568F1E8
:1015D000EFE0E61750F14115510539F1FA0101909C
:1015E0000020E9F731970E2F041B013108F000E1CC
:1015F0006C2D8D2D0E945E0A5701002361F0102F83
:101600008881F50181935F018991682F82E00E94B2
:10161000B60B1150A9F7F701D08AC18A028B64EF8B
:1016200071E081E79AE00E94970ADF91CF911F91C4
:101630000F91FF90EF90DF90CF90BF90AF90089503
:10164000CF93DF93CDB7DEB7A0970FB6F894DEBF88
:101650000FBECDBF282FDE01119690E0FA014F5F3B
:101660005F4F8491882321F08D939F5F9F31B0F36A
:101670001C92AE014F5F5F4F822F0E94D00AA0964E
:101680000FB6F894DEBF0FBECDBFDF91CF910895A6
:101690008091330390913403892BA9F160912D033C
:1016A00070912E0380912F03909130030E940707C1
:1016B000882349F180912C03E0913303F0913403A6
:1016C0008170099580912C0391E0892780932C03E8
:1016D00080913103909132039C01442755278091DA
:1016E000030390910403A0910503B0910603820FB8
:1016F000931FA41FB51F80932D0390932E03A093D7
:101700002F03B0933003089508951092340310927C
:10171000330381E00E94540A08950F931F93CF93DF
:10172000DF93EB018830C0F4992723E0880F991FDD
:101730002A95E1F780640E94540A07E010E0FE0158
:10174000219684910E94250A0150104017FFF7CF7F
:1017500060E0862F0E945E0ADF91CF911F910F916A
:101760000895813308F080E381BF08958230D1F479
:1017700067FF15C0643E31F0663F41F06C3F51F0A9
:10178000643C11F461EE0BC0663D11F46FEE07C0CE
:101790006C3D11F465EF03C06F3D09F462EE862FD6
:1017A0000E94250A089508951F93CF93DF93182F61
:1017B000EB01FB016491662349F0812F0E94B60B77
:1017C0002196FE018491682F8823B9F7DF91CF918C
:1017D0001F9108951F93CF93DF93182FEB018881FA
:1017E000882341F08991682F812F0E94B60B888150
:1017F0008823C1F7DF91CF911F9108951F93CF9355
:10180000DF93CDB7DEB7C055D0400FB6F894DEBF3A
:101810000FBECDBF67961FAD679769968EAD9FAD22
:101820006997AE01475A5F4FBC01CE0101960E94F5
:101830005822BE016F5F7F4F812F0E94EA0BC05B71
:10184000DF4F0FB6F894DEBF0FBECDBFDF91CF9153
:101850001F9108951F93CF93DF93CDB7DEB7C05587
:10186000D0400FB6F894DEBF0FBECDBF67961FAD58
:10187000679769968EAD9FAD6997AE01475A5F4FE6
:10188000BC01CE0101960E948122BE016F5F7F4F95
:10189000812F0E94EA0BC05BDF4F0FB6F894DEBFCA
:1018A0000FBECDBFDF91CF911F910895823019F403
:1018B0000E940A0A08958FEF9FEF08950895E82F78
:1018C000FF27EF70F070E25EFD4F84919927089535
:1018D00089E691E008958091770182FF05C08091AB
:1018E0006B0190916C0108958091690190916A015A
:1018F000089508958091770182608093770108951B
:101900000F931F93CF93DF93C9E6D1E080917701C6
:1019100099278C010170107080FF03C080E090E077
:1019200021C060916F01709170018091710190915F
:101930007201611571058105910531F00E9407075B
:10194000882311F4C8010EC01A821B821A8A1B8ACE
:1019500010926A01109269011E861C8A0E94450439
:1019600081E090E0DF91CF911F910F9108959C014C
:1019700080916B0190916C01892B11F4C90108953C
:101980002F703F7B77FD3064CB018F70907044E007
:10199000880F991F4A95E1F7822B932B089508959C
:1019A000FC018091690190916A0120916B01309155
:1019B0006C01E817F907F9F460937901232BB1F072
:1019C00080916D0190916E01F4E096958795FA955E
:1019D000E1F7BC016F707070892F99278695869505
:1019E00080FD7068CA010E94B70C0FC050936E0151
:1019F00040936D010EC0E217F30769F4BA018091BC
:101A00006D0190916E010E94B70C90936E018093CE
:101A10006D010E944504089508959C01892B69F485
:101A20001092770110926F01109270011092710163
:101A3000109272010E94800C089560937901509376
:101A40006E0140936D018091030390910403A09176
:101A50000503B091060388519C4FAF4FBF4F816083
:101A600080936F0190937001A0937101B093720104
:101A70008091770182FF09C081608B7F809377011D
:101A800030936C0120936B0107C08E7F80937701A8
:101A900030936A01209369010E94450408950895D6
:101AA000209177012B7F21602093770190936C0127
:101AB00080936B0180916D0190916E010E94B70C33
:101AC00090936E0180936D010E9445040895CF9319
:101AD000DF93EB01809378010E945F0C80937A0181
:101AE000209759F04DE751E060E070E0CE010E9490
:101AF0003521D0937C01C0937B010E944504DF9186
:101B0000CF910895CF93C82F882319F06EE571E027
:101B100002C06EE771E084E00E948D0BCC2319F0C7
:101B200066E571E002C066E771E085E00E948D0B1A
:101B3000CC2319F06EE471E002C06EE671E086E03D
:101B40000E948D0BCC2319F066E471E002C066E6BA
:101B500071E087E00E948D0BCF910895CF93DF93C2
:101B6000C82FDD27C4FF02C083E001C085EA0E94C0
:101B7000250AC0FF02C084E001C085EA0E94250A50
:101B8000C1FF02C085E001C085EA0E94250AC2FFAC
:101B900002C086E001C085EA0E94250AC3FF02C098
:101BA00087E001C085EA0E94250ADF91CF91089560
:101BB000809389010E9445040895882319F066E204
:101BC00071E002C06EE271E082E00E948D0B089528
:101BD0000895882319F066E371E002C06EE371E0B6
:101BE00081E00E948D0B089508950F931F93CF936A
:101BF00009E611E0C0918901CC2399F060E081E011
:101C00000E945E0A8C2F81500E94F61ABC0182E06D
:101C10000E94D40B1092890188EE93E00E94DD08A7
:101C200002C0882319F00E94850B03C0682F0E9410
:101C30005E0A8091690190916A01892BF9F00E94F6
:101C4000741BFC01828193814091690150916A016A
:101C50008417950749F42185328580917B01909105
:101C60007C012817390751F04283538380917B010F
:101C700090917C01818792870E94191B20916901B4
:101C800030916A012115310529F4F8012483358347
:101C9000108A17868091770182FD0DC080917301B3
:101CA00090917401A0917501B09176010097A10502
:101CB000B10519F105C06EE272E082E00E94D40B1A
:101CC0008091730190917401A0917501B09176019A
:101CD000BF93AF939F938F9381E392E09F938F93F2
:101CE00082E08F930E942A0C8DB79EB707960FB69D
:101CF000F8949EBF0FBE8DBF43C02115310531F44E
:101D000064E472E082E00E94D40B18C03F932F93EA
:101D10008BE492E09F938F93C2E0CF930E942A0CB2
:101D2000809177010F900F900F900F900F9080FF90
:101D300002C08C2F01C080E20E94250AC091780168
:101D40000E946D04853010F085E00EC0833061F490
:101D50008C2F99278370907023E0880F991F2A9504
:101D6000E1F782539E4F08C0992703E0880F991F1F
:101D70000A95E1F782519E4FBC0182E00E94D40B8C
:101D80006CE080E00E945E0A8091790199278F774C
:101D900090709F938F9380E592E09F938F9382E062
:101DA0008F930E942A0C80917801992783709070FC
:101DB0000F900F900F900F900F90019779F483E19F
:101DC0000E945909882331F080E00E94250A6EE0C4
:101DD00071E010C080E20E94250A0FC080E00E94DE
:101DE000250A8091790187FF03C066EC71E002C08B
:101DF0006EEB71E080E00E948D0B0E946D04C82F95
:101E0000813049F488E00E94C11AAC0160E08C2F57
:101E10000E94200BE0C040E050E060E0862F0E946E
:101E2000D00AC0E08AE00E945909882371F08091AD
:101E30006B0190916C01892B39F48091780199277D
:101E400083709070039709F4C1E060E081E00E9424
:101E50005E0A8091730190917401A0917501B09117
:101E600076010097A105B10509F442C08DE00E94FA
:101E70005909882329F48EE00E945909882381F1A9
:101E800084E592E09F938F93C2E0CF930E942A0C47
:101E90008DE00E9459090F900F900F90882379F0E0
:101EA00066E371E081E00E948D0B6EE271E08C2FA1
:101EB0000E948D0B6CE271E089EE9DE00EC06EE336
:101EC00071E081E00E948D0B66E271E08C2F0E9430
:101ED0008D0B6CE271E08DED9DE00E94970A7BC056
:101EE00086E00E94C11ABC0182E00E94D40B44C06B
:101EF00080916B0190916C01009769F19F938F9392
:101F000080E692E09F938F9382E08F930E942A0C49
:101F100080916D0190916E0114E0969587951A95C8
:101F2000E1F7282F2F70892F9927869586950F9096
:101F30000F900F900F900F9080FD2061822F0E94D4
:101F4000AE0DCC2321F08CE30E94250A15C080E25F
:101F50000E94250A2CC08DE791E09F938F9385E620
:101F600092E09F938F9382E08F930E942A0C0F90B0
:101F70000F900F900F900F90CC23C9F080916B01C0
:101F800090916C01892B99F480916D0190916E0173
:101F9000A4E096958795AA95E1F78F7080610E94DD
:101FA000AE0D81E00E94820D66E871E011C02091C3
:101FB0006D012F7080916D0190916E0197FD2061F0
:101FC000822F0E94AE0D80E00E94820D6EE871E0CB
:101FD00083E00E948D0BCF911F910F910895609126
:101FE0006F01709170018091710190917201611582
:101FF00071058105910561F00E940707882341F072
:1020000010926F0110927001109271011092720182
:1020100008950895AF92BF92CF92DF92EF92FF9210
:102020000F931F93CF93DF93CDB7DEB72C970FB6E7
:10203000F894DEBF0FBECDBF8C0129E6C22E21E091
:10204000D22E86E0FE01319611928A95E9F7013190
:102050001105DCF40F3011050CF0EFC00A3011054A
:1020600009F415C20B3011053CF40115110509F4F2
:1020700010C117FD1BC220C10C30110509F460C04E
:102080000D3011050CF07BC048C105311105C1F1BF
:10209000063111057CF40231110509F4EAC0023160
:1020A00011050CF4E8C003311105B9F10431110533
:1020B00091F0FCC10F3811054CF40D3811050CF0EE
:1020C0005EC00A38110509F4EFC1F0C103391105EA
:1020D00009F4EAC1EBC18091790199278F7790705B
:1020E00020917A013327821793070CF0DFC10E94F9
:1020F0006D04833009F0DAC1809179018F5F1DC0D2
:1021000020917901822F99278F779070892B09F47C
:10211000CDC1215020937901C7C1809178019927C1
:1021200083709070019729F46EE071E080E00E9466
:102130008D0B809179018095807880937901B4C16D
:102140008AE00E945909882399F080916B0190914F
:102150006C01892B69F080916D0190916E0120E0F6
:1021600030E48227932790936E0180936D019CC188
:1021700080916D0190916E0120E030E874C086E09E
:1021800097E0A92EB12CAC0EBD1EF50111928A95D7
:10219000E9F78091730190917401A0917501B0915C
:1021A00076010097A105B10509F445C0E0907301DF
:1021B000F09074010894E108F108EE0CFF1CC801CE
:1021C0008F7790700E9721F481E090E0E82AF92A49
:1021D00007FF16C01A8660E070E0CB010E94970AE4
:1021E0006EE971E081E00E948D0B66EA71E082E0A9
:1021F0000E948D0BF601128613861486158602C086
:1022000081E08A878E2D8F778F83EE0CEF2CEE1C6A
:10221000FF08F1948E2D8F778887EE0CEF2CEE1C43
:10222000FF08F1948E2D83708987A50166E080E018
:102230000E94BB1D39C107FD37C1A3EFFA2EF00E76
:102240008AE00E945909882319F0F7EFFF2EF00E5B
:1022500021E030E002C0220F331FFA94E2F78091B0
:102260006D0190916E0182279327F60184839583F7
:102270001BC143E006C08AE00E945909882321F06F
:1022800042E060E280E002C0482F60E20E942F201E
:102290000BC18091730190917401A0917501B0916F
:1022A00076010097A105B10539F48FEF0E948F1ACE
:1022B00081E00E94F50DFAC0809173019091740144
:1022C000A0917501B09176019C01AD01E3E0220F70
:1022D000331F441F551FEA95D1F7280F391F4A1F96
:1022E0005B1F280F391F4A1F5B1FC801AA2797FDD4
:1022F000A095BA2F280F391F4A1F5B1F2030F8E224
:102300003F07F0E04F07F0E05F070CF0CFC0F601A9
:102310002287338744875587C7C079E6E72E71E067
:10232000F72E86E0AE01495F5F4FFA0111928A9560
:10233000E9F70091730110917401209175013091BA
:10234000760160916B0170916C01011511052105F9
:10235000310509F48FC06115710581F1A090690103
:10236000B0906A01C501AA27BB2780179107A20771
:10237000B30741F0CB01AA27BB2780179107A2071B
:10238000B307E1F4809177018E7FF6018687809113
:1023900069018F778F83AA0CAB2CAA1CBB08B19460
:1023A0008A2D8F77888765E080E00E94BB1DF6014B
:1023B0001282138210926A01109269018091690160
:1023C00090916A019C014427552780917301909157
:1023D0007401A0917501B091760160917701281781
:1023E00039074A075B0731F481E068276B7FF70103
:1023F000668748C06C7FF7016687128A138A148A41
:1024000060917D0181E00E945E0A80E00E94C11A15
:10241000BC0182E00E94D40B8091770199279695A8
:102420008795969587959C012170307080FD12C02C
:10243000F701228333832483358330936A01209309
:102440006901178660917301709174018FEF0E948A
:10245000EB1B0BC0409173015091740160916901B5
:1024600070916A018FEF0E941A1C809177018B7F17
:10247000F70106C0672B29F4809177018460F6018B
:102480008687F70112861386148615860DC0109272
:10249000730110927401109275011092760180916F
:1024A00077018B7F809377010E9445042C960FB6AD
:1024B000F894DEBF0FBECDBFDF91CF911F910F917A
:1024C000FF90EF90DF90CF90BF90AF900895FB0109
:1024D00021E057FF04C020E0509541955F4F8330C5
:1024E000910549F18430910534F48130910591F0E2
:1024F000029729F12AC08430910519F0059761F0FF
:1025000024C081818F5F8183992784179507ECF020
:10251000222359F0118219C081818150818399272A
:102520008417950794F0222321F0842F8150818312
:102530000CC021830AC012821382168A06C090E062
:102540008281882309F491E0928380E090E00895ED
:102550000F931F93CF93DF938C010E946B0CEC01C0
:10256000009731F469E375E082E00E94D40B0FC05C
:102570009F938F938FE395E09F938F9382E08F9348
:102580000E942A0C0F900F900F900F900F90011542
:10259000110521F0B80182E00E94D40BCE01DF9139
:1025A000CF911F910F9108950F931F93CF93DF93B6
:1025B000EC018B01009731F097FD35C0029702972F
:1025C00090F52BC060E081E00E945E0AF8018281F4
:1025D000882359F463E475E082E00E94D40B6CE434
:1025E00075E082E00E94D40B18C00E947C1BDC01C5
:1025F000CB01BF93AF939F938F9382E595E09F9319
:102600008F9382E08F930E942A0C8DB79EB7079616
:102610000FB6F8949EBF0FBE8DBF40E050E0B801EA
:10262000CE010E94671280E090E0DF91CF911F9170
:102630000F9108958230910541F08330910541F466
:1026400040E050E00E94671203C08FEF9FEF0895B3
:1026500080E090E0089508952F923F924F925F920C
:102660006F927F928F929F92AF92BF92CF92DF92A2
:10267000FF920F931F93CF93DF93CDB7DEB72697CB
:102680000FB6F894DEBF0FBECDBF8C015B010E9478
:10269000680C6C010230110509F457C003301105B4
:1026A0003CF401151105E9F00130110531F0CAC003
:1026B000063011050CF0C6C02CC0FC01F7842F2D8C
:1026C000269526952370F3E0FF2211F451E0F52EB4
:1026D00083E0F89EC0011124280F2350F5012183C7
:1026E000B1C060E081E00E945E0A8EE595E00E9444
:1026F000A812892B09F4A6C0F50191818AE0989F60
:10270000C001112481569D4FBC0182E00E94D40B70
:1027100099C049E050E0B501C8010E946712F60176
:10272000808191818F3F910509F008F48BC0F501FC
:102730008181882311F486E08183F50181818630CF
:1027400008F080C088E081837DC0FC014280538016
:102750004114510409F076C0F5018281882309F4FF
:1027600069C0F601808091808114910409F46AC0E7
:10277000F5012181822F63E00E949D25F82EF394BC
:10278000822F0E949D25892F9927880F991F880FD6
:10279000991FF82AF6012288338834E1632E712CC0
:1027A0006C0C7D1C8501065F1F4FB301C8010E94A0
:1027B000512286E0FE01319611928A95E9F7882D23
:1027C0008F778983C401880F892F881F990B919572
:1027D0008F778A83FFE7FF22FB82AE014F5F5F4F57
:1027E00064E08FEF0E94BB1D60E081E00E945E0A02
:1027F00080E00E94C11ABC0182E00E94D40BA201B9
:1028000060E0C2010E940D0DB4018FEF0E94EB1B2E
:10281000B801C3010E9451222114310459F09301DF
:10282000F601478560817181C1010E947820F6011F
:10283000828B938B90E0F5018281882309F491E0EB
:10284000F501928380E090E026960FB6F894DEBF03
:102850000FBECDBFDF91CF911F910F91FF90DF9001
:10286000CF90BF90AF909F908F907F906F905F9030
:102870004F903F902F900895482F30E0832F992755
:1028800087FD9095FC01E259FD4F2491241729F012
:102890003F5F222399F78FEF9FEF08950895EF92FE
:1028A000FF920F931F93CF93DF93EB01823091053B
:1028B00009F486C08330910534F4009709F43EC0D2
:1028C000019769F0BAC08430910509F443C084309F
:1028D00091050CF470C0059709F456C0AEC00E9473
:1028E000680C8C01FC0180819181892B09F4A5C0C1
:1028F00064E1E62EF12CE00EF11E8E01065F1F4F03
:1029000065960C171D07B8F4F7018081882339F00C
:102910000E943C1487FD03C0F701808101C080E262
:10292000F80181938F01F7018081882351F3089486
:10293000E11CF11CE6CFF80110827FC00E94A812B2
:1029400060E081E00E945E0A2A96BE0182E00E9459
:10295000EA0B73C08981FB01E80FF11DEF012A9694
:1029600082850E943C148F5FE82FFF27E7FDF095DA
:10297000E259FD4F8491882319F4EEE6F2E0849148
:10298000992787FD909515C08981FB01E80FF11DFE
:10299000EF012A9682850E943C14181614F08FE2EB
:1029A00001C08150E82FFF27E7FDF095E259FD4F68
:1029B0008491888342C049E050E00E9467123DC084
:1029C0000E94680C8C01FC0182819381892BA9F5FE
:1029D0009A81992349F489E08B8381E0888F9983D8
:1029E0009F8B8A838E8B29C089818F5F89838F8B90
:1029F0008B3018F11B821A821E8A8CE098012C5EA3
:102A00003F4FD901FE013A9601900D928A95E1F768
:102A1000F80182899389009731F04785608171813F
:102A20000E94782007C0A901F80167858081918103
:102A30000E942D21F801828B938B80E090E0DF9142
:102A4000CF911F910F91FF90EF9008958F929F92D9
:102A5000BF92CF92DF92EF92FF920F931F93CF938B
:102A6000DF93CDB7DEB727970FB6F894DEBF0FBE62
:102A7000CDBF9C018B018230910509F455C0833094
:102A800091052CF40097C1F0019759F0C8C084302B
:102A90009105D9F1843091050CF441C00597C9F135
:102AA000BEC04BE050E060E270E0C8010A960E94B0
:102AB0004A22F801158AB3C0FB018281882309F4F8
:102AC000AEC08181882309F4AAC0065F1F4FA80108
:102AD000B90199270E9435219F938F9381E695E054
:102AE0009F938F93F2E0FF2EFF920E942A0C60E0EA
:102AF00081E00E945E0AB8018F2D0E94EA0B0F90C0
:102B00000F900F900F900F908AC0FB018181992741
:102B100021C0FB01818199270E9422221DC049E02A
:102B200050E00E9467127BC090E0FB018281882305
:102B300009F491E0F80192830E94680C7C01F8018D
:102B4000B280BB2061F0FC0182899389009711F06B
:102B5000828902C00E941E22F801818360C0EAE0DF
:102B60008E2E912C800E911EF8018181A401BE0150
:102B7000695F7F4F99270E9435216C01F70112820E
:102B8000138210821182BC018FEF0E94EB1BF701B0
:102B900080819181892B81F186E0FE01319611922D
:102BA0008A95E9F78C2D8F778983C601880F892F45
:102BB000881F990B91958F778A838F818F778B836D
:102BC000AE014F5F5F4F64E08FEF0E94BB1D6B2D26
:102BD00081E00E945E0A8B2D0E94C11ABC0182E036
:102BE0000E94D40B40E050E06B2DCA010E940D0DF5
:102BF000B6018FEF0E94EB1BF70180819181892B39
:102C000059F0B401C70144960E945122F801818114
:102C10009927F701828B938B8FEF9FEF02C080E0A3
:102C200090E027960FB6F894DEBF0FBECDBFDF91C0
:102C3000CF911F910F91FF90EF90DF90CF90BF90B9
:102C40009F908F9008950F931F93CF93DF93EC0184
:102C50000E94680C8C01209719F02297C9F03DC0A2
:102C6000CE010E94A812892BC1F160E081E00E9490
:102C70005E0AF80182899389892B11F081E001C0F5
:102C800082E00E94C11ABC0182E00E94D40B25C0E0
:102C9000FC01C281D381209701F580819181892B2C
:102CA000E1F082899389892BC1F060E081E00E9484
:102CB0005E0A83E00E94C11ABC0182E00E94D40B2C
:102CC00084EF91E00E94DD08F801828993890E94D7
:102CD0004E20F801C28BD38B148A80E090E0DF9104
:102CE000CF911F910F9108951F93CF93DF93EB0125
:102CF0008230910509F440C0833091052CF400978F
:102D000089F0019731F04CC0863091050CF048C035
:102D10002EC00E94741BFC01848163E00E949D25EB
:102D200089833EC060E081E00E945E0A898113E0F1
:102D3000819F802D11240E94B10B82E090E00E94BF
:102D4000DD0881B7612F0E949D25898399279F9374
:102D50008F9385E695E09F938F9382E08F930E94F7
:102D60002A0C0F900F900F900F900F9019C04FEEFC
:102D70005FEF0E94671214C08A81882359F00E9475
:102D8000741B398123E0329F90011124FC012483BC
:102D90000E94191B90E08A81882309F491E09A83AC
:102DA00080E090E0DF91CF911F910895EF92FF9224
:102DB0000F931F93CF93DF93CDB7DEB726970FB650
:102DC000F894DEBF0FBECDBF8C017B010E94680C62
:102DD000DC018D919C911197892B39F0FD0187853C
:102DE000992783709070039731F060E081E00E9432
:102DF0005E0A85E03AC00230110509F4A3C0033031
:102E000011053CF40115110539F10130110571F07E
:102E1000F8C00430110509F493C0043011050CF416
:102E2000EAC00530110509F4E2C0EBC08EEF9FEF58
:102E3000F701818F928F2091910130919201C90108
:102E400001978050944020F4F70124833583D9C042
:102E5000F70104831583D5C060E081E00E945E0A1B
:102E6000F7018281882341F487E00E94C11ABC01E6
:102E700082E00E94D40BC5C060E081E00E945E0A3F
:102E8000F701848195819F938F9389E695E09F93C5
:102E90008F9312E01F930E942A0C0F900F900F90B7
:102EA0000F900F90F7018381843059F48FE695E0FD
:102EB0009F938F931F930E942A0C0F900F900F9057
:102EC00011C0F701808599279F938F9383E795E041
:102ED0009F938F931F930E942A0C0F900F900F9037
:102EE0000F900F90F701818D928D97FD03C067E7DA
:102EF00075E00AC08E5F9F4F19F46FE775E004C05C
:102F000084E00E94C11ABC0182E00E94D40B81E0DF
:102F1000F701808F868B83819927813091056CF032
:102F20008330910524F00497029738F402C083E0BF
:102F300001C088E0F701878B64C0F701168A61C081
:102F400084E056C0F701828124813581882389F489
:102F500041E0438380E094E0868397838217930760
:102F60002CF481E090E0F70184839583F70142839C
:102F700048C0309392012093910121153105B9F198
:102F8000F70183818150823090F18C918F77898312
:102F90008D919C91880F892F881F990B91958F7720
:102FA0008A83848181508F778B8321503040220F18
:102FB000232F221F330B322F37702085822F992722
:102FC0008078907095958795382B3C832F772D834B
:102FD0001E82AE014F5F5F4F67E08FEF0E94BB1D07
:102FE000F70113820E946D0A8FEF9FEF0CC081E002
:102FF000F701838306C040E050E0B701C8010E949A
:10300000671280E090E026960FB6F894DEBF0FBE00
:10301000CDBFDF91CF911F910F91FF90EF90089559
:10302000CF92DF92EF92FF920F931F93CF93DF9394
:103030007C01C62F0E94850B0E94741B6C01CA3054
:1030400008F06FC085E0C89F800111240E5F1E4FFD
:10305000F7018281882311F080E001C082E00E94A4
:10306000250AF6018581992781309105B1F08230DA
:1030700091051CF4892B39F031C082309105B9F0EB
:103080000397F9F02BC08C2F992754E0880F991FD4
:103090005A95E1F787559B4F1DC08C2F992744E027
:1030A000880F991F4A95E1F7875E9B4F13C08C2FBD
:1030B000992734E0880F991F3A95E1F787579C4F7D
:1030C00009C08C2F992724E0880F991F2A95E1F7D2
:1030D00087509D4FBC0182E00E94D40BE8018C8197
:1030E00087FD0BC060E081E00E945E0A8C810E9437
:1030F000C11ABC0182E00E94D40BE801EA81FB8185
:10310000309721F0B70180E090E00995F7018689BA
:10311000882329F06789808D0E94670A02C00E9477
:103120006D0ADF91CF911F910F91FF90EF90DF908B
:10313000CF90089560E0E2E0F1E0482F552747FD89
:10314000509520E030E0808199278417950711F48D
:10315000C90108956F5F2F5F3F4F3596693098F32F
:103160008FEF9FEF08950895BF92CF92DF92EF9275
:10317000FF920F931F93CF93DF93CDB7DEB76B977B
:103180000FB6F894DEBF0FBECDBFB82E28E02817CB
:1031900018F480E090E0B3C16E010894C11CD11C0A
:1031A0008BE1F60111928A95E9F7A89585E0B89E22
:1031B000F0011124EE5FFE4F0280F381E02D309785
:1031C00021F0B60181E090E009956B2DC6010E94C7
:1031D00010180E94710415E0B19E7001112482E064
:1031E00091E0E80EF91E0E940A0AAC018B309105AD
:1031F00009F497C08C30910534F497FDEACF0A9713
:103200000CF4FEC0D6C08331910509F48AC0843124
:10321000910524F4419709F46BC1DBCF843191050A
:1032200019F0459751F1D5CFF6018281882381F0BD
:10323000F701228133812115310531F0BE016F5F25
:103240007F4F84E090E051C1F60181818F5F28C0FB
:10325000F601868BF7019081F7E0FB1534F0F7015A
:103260008581891711F4B39431C0892F0E949A186F
:10327000682F772767FD709540C0F601828188230B
:1032800089F0F701228133812115310531F0BE012A
:103290006F5F7F4F85E090E028C1F601818181500A
:1032A000818329C1F601868B6B2DF7019081BB20AC
:1032B00091F02BEF3FEFE20EF31EF701808125E046
:1032C00030E0E20EF31E891731F4BA946B2D7727A4
:1032D00067FD709512C037E03B1564F0D701159675
:1032E000F7018581891731F46F5F68301CF41596FA
:1032F0008C91F8CF772767FD7095B62E85E0689F93
:10330000F0011124EE5FFE4F0280F381E02D309733
:1033100009F4F1C0BE016F5F7F4F81E090E0099535
:10332000EAC0F7019181992361F1092F112706570E
:103330001E4FF801808118162CF0892F0E949A18D0
:10334000F8018083F7018181E82FFF27E657FE4FC0
:1033500080810E94B418282F332727FD3095F7016C
:103360008181E82FFF27E657FE4FC90137FF04C0D0
:1033700088279927821B930B808337FFBCC0B194A9
:103380003AC0F701228133812115310551F0BE0188
:103390006F5F7F4F82E090E0F901099599237CF3FC
:1033A00019C0F6018281882309F491E0F601928325
:1033B000A2C0F60182818823F1F0F70122813381D6
:1033C00021153105A9F0BE016F5F7F4F83E090E0CA
:1033D000F9010995F6018281882309F08CC0F70173
:1033E00022813381BE016F5F7F4F81E090E07DC01D
:1033F000F601128280C08B2D992787FD90957FC0A2
:10340000F601838199278430910509F446C08530FF
:1034100091054CF48230910539F18330910584F4A3
:10342000019771F068C08830910551F0893091059D
:103430001CF40597A9F15FC0099709F444C05BC06B
:10344000F60186819781892B21F48FEF9FE7868390
:103450009783F60186819781841795070CF44BC0FA
:103460001482158282E08383F601848195819C0118
:1034700063E0220F331F6A95E1F7280F391F280FE9
:10348000391F240F351F37FD36C08681978182177B
:1034900093078CF1248335832EC0F60110861383A5
:1034A000F60190858AE0989F90011124240F351F22
:1034B0002F3F310509F008F420878EEF9FEFF601CA
:1034C000818F928F18C0F6018181E80FF11D842F42
:1034D000805D8287F701228133812115310559F002
:1034E000BE016F5F7F4F82E090E0F901099503C054
:1034F00080E00E9449046B2DCE01019668CE6B9648
:103500000FB6F894DEBF0FBECDBFDF91CF911F91F4
:103510000F91FF90EF90DF90CF90BF900895CF93E1
:10352000C82F66E071E080E00E948D0B6EE071E0D4
:1035300082E00E948D0B80918A01893010F01092F8
:103540008A01C7FD04C08C2F0E94B4180EC0809160
:103550008A010E94B418992787FD909597FF03C0B0
:10356000909581959F4F80938A0166EC71E080E091
:103570000E948D0B66EA71E082E00E948D0BCF9174
:103580000895CF93C82F893018F08FE298E02CC0AF
:103590000E94741BFC01858199278230910581F07E
:1035A000833091051CF4019721F018C0039779F03E
:1035B00015C081E1C89FC00111248A56984F14C0DC
:1035C00081E1C89FC00111248350994F0DC081E152
:1035D000C89FC00111248C59994F06C081E1C89F32
:1035E000C001112485539A4FCF910895882319F073
:1035F0008CE398E008950E94741BFC018581992753
:103600008230910561F0833091051CF4019721F01F
:103610000CC0039739F009C08AEB95E0089589EA58
:1036200095E0089588E995E0089587E895E0089584
:103630000895EF92FF921F93CF93DF9383E9E82ED3
:1036400081E0F82EC0E0D0E01FE1CE010E942622EA
:10365000F70161917F01861719F0CE010E943F2288
:10366000A8951150219617FFF0CFDF91CF911F91B0
:10367000FF90EF90089590919801943008F091E0B8
:103680008FE0E3E9F1E011928A95E9F788E1809310
:103690009701909398010E94191B089540E250E011
:1036A00060E070E083E991E00E942E228091950114
:1036B000909196018F5F9F4F11F40E943B1B809168
:1036C0009801843010F0109298018AEF9FEFA1E0EA
:1036D000B0E0ABBFFC0187918F3F21F0882311F050
:1036E00080936F000895089583E991E00895809391
:1036F00098010E94191B08958CEF9FEFA1E0B0E0A4
:10370000ABBFFC0187919791A791B691B070BC01B6
:10371000CD0108958FEF9FEFA1E0B0E0ABBFFC01BA
:10372000879199270895FC01868599279695879515
:103730009C012170307080FD02C0C9010895808114
:103740009181009711F081E090E008950895FC01C7
:1037500082819381009711F081E090E008950895AF
:10376000CF92DF92EF92FF920F931F93CF93DF934D
:10377000C82E7B01EA010E94680C8C01209711F190
:10378000DD24A7016C2D80E00E94BB1D8AE08093A0
:10379000350302C00E947104C801FE010995882307
:1037A00021F4809135038823A9F70E94E31C81113D
:1037B000DD24C801FE010995882321F4D39487E014
:1037C0008D15F8F6DF91CF911F910F91FF90EF903B
:1037D000DF90CF900895CF93DF93CDB7DEB72697D4
:1037E0000FB6F894DEBF0FBECDBF61157105C9F0ED
:1037F00086E0FE01319611928A95E9F7862F8F7740
:103800008983660F672F661F770B7195862F8F77D9
:103810008A8343E95BE1BE016F5F7F4F81E00E94D5
:10382000B01B26960FB6F894DEBF0FBECDBFDF915A
:10383000CF910895CF93DF93CDB7DEB726970FB61C
:10384000F894DEBF0FBECDBF6115710539F141158A
:10385000510521F186E0FE01319611928A95E9F732
:10386000862F8F778983660F672F661F770B719579
:10387000862F8F778A83842F8F778B83440F452FF2
:10388000441F550B5195842F8F778C8347EA5BE15A
:10389000BE016F5F7F4F82E00E94B01B26960FB67D
:1038A000F894DEBF0FBECDBFDF91CF910895F8949D
:1038B000FFCFFC0180E0482F57E02191282780E0CE
:1038C000922F96958F5F20FF03C0292F252701C0D7
:1038D000292F8830A8F33327822F4F5F483068F3B1
:1038E00027FD8095992708950F931F938C010E94BF
:1038F000591CF8019085891719F080E090E002C00A
:1039000081E090E01F910F910895EF92FF920F9345
:103910001F93CF93DF93CDB7DEB729970FB6F894F7
:10392000DEBF0FBECDBF9C0180912F0180687E015C
:103930000894E11CF11C898383E0F70181838701EE
:103940000E5F1F4F822F8F77F8018193220F232F55
:10395000221F330B3195822F8F778193862F8F779C
:1039600081938F01CA01892F9927869586958F7338
:10397000808367FF02C0806480830F5F1F4FCA018E
:1039800023E0969587952A95E1F78F77F801819343
:10399000842F8295807F8F7781938F01C7010E944A
:1039A000591CF8018083C7010E94B90629960FB6F9
:1039B000F894DEBF0FBECDBFDF91CF911F910F9165
:1039C000FF90EF9008958091B301882319F480E06F
:1039D00090E008951092B30181E090E00895089579
:1039E000EF92FF920F931F93CF93DF93CDB7DEB784
:1039F00029970FB6F894DEBF0FBECDBF0E947C1B87
:103A00007B018C0165C0A8958A81843009F060C073
:103A1000CE0101960E94741C882309F459C0D80174
:103A2000C7018F779070A070B0702E813327442724
:103A3000552782179307A407B50709F049C0D80195
:103A4000C70180789F73A070B07027E0B595A795E7
:103A5000979587952A95D1F72D81332744275527A8
:103A600082179307A407B50799F5D801C70180709D
:103A7000907CAF71B070FEE0B595A795979587954E
:103A8000FA95D1F72C8133274427552782179307BE
:103A9000A407B507E9F4D801C70180709070A07E33
:103AA000B070E5E1B595A79597958795EA95D1F71B
:103AB0002B8133274427552782179307A407B5077F
:103AC00039F489818F7780932F0181E090E007C0DE
:103AD000CE0101960E94C306009709F094CF299663
:103AE0000FB6F894DEBF0FBECDBFDF91CF911F910F
:103AF0000F91FF90EF90089580912F0199270895DD
:103B00000F931F93CF93DF93CDB7DEB729970FB6EF
:103B1000F894DEBF0FBECDBFFA01A89580912F01AA
:103B2000806889836A838E010D5F1F4F95E030970F
:103B300029F081918F77D8018C9302C0D8011C9213
:103B400091500F5F1F4F97FFF2CFCE0101960E9459
:103B5000591CF8018083CE0101960E9485069927A1
:103B600029960FB6F894DEBF0FBECDBFDF91CF917F
:103B70001F910F9108950F931F93CF93DF93082FF9
:103B8000162FEA0102C00E947104AE01612F802F3E
:103B90000E94801D8823B9F3DF91CF911F910F916F
:103BA00008959F92AF92BF92CF92DF92EF92FF92D1
:103BB0000F931F93CF93DF93CDB7DEB72F970FB639
:103BC000F894DEBF0FBECDBF31C2CE0101960E9478
:103BD000741C882309F42AC26E010894C11CD11CEC
:103BE0000E94680C5C01F6016181862F9927AA2743
:103BF000BB27FC013397E032F10508F0EDC1EA5B29
:103C0000FF4FEE0FFF1F0590F491E02D0994F60190
:103C100082810E944904E0C1F6018281282F332766
:103C2000838199279695982F882797958795282B94
:103C3000392BD5018D919C918217930709F0CCC146
:103C40000E94800CC9C1F6018281A82FBB27838105
:103C500099279695982F882797958795A82BB92B04
:103C60008581282F3327A901542F4427550F550F3D
:103C7000868199278F77907013E0880F991F1A9586
:103C8000E1F7482B592B878199278077907074E052
:103C9000959587957A95E1F7482B592B683029F44B
:103CA000BA01CD010E94500D97C1F601648126FD35
:103CB0006068CD010E940D0D8FC1F6018581282F0E
:103CC0003327868199279695982F882797958795EA
:103CD000282B392BB90184810E94670D7DC10E9478
:103CE0007A0C7AC1F6018281A82FBB27838199279C
:103CF0009695982F882797958795A82BB92B85811E
:103D0000282F3327A901542F4427550F550F86819B
:103D100099278F77907003E0880F991F0A95E1F734
:103D2000482B592B878199278077907014E09595BF
:103D300087951A95E1F7482B592B648126FD606819
:103D4000CD010E94D00C48C1F50182899389892B4D
:103D500041F0A8E09A2E82898F778A878289938999
:103D600007C09924D5018C918F778A878D919C917A
:103D7000880F892F881F990B91958F778B87F50175
:103D8000868580FF02C0F0E19F2A0E947C1B7B0198
:103D90008C01862F8F778C8767E016950795F794AF
:103DA000E7946A95D1F78E2D8F778D8757E016951A
:103DB0000795F794E7945A95D1F78E2D8F778E87D4
:103DC00047E016950795F794E7944A95D1F78E2D1D
:103DD000877089298F87AE01465F5F4F6BE08FEF59
:103DE0000E94BB1DF9C00E947C1B7B018C01DC0181
:103DF000CB018F779070A070B070F60124813327CB
:103E00004427552782179307A407B50709F00EC169
:103E1000D801C70180789F73A070B07037E0B69565
:103E2000A795979587953A95D1F72581332744270C
:103E3000552782179307A407B50709F0F7C0D801E3
:103E4000C7018070907CAF71B0702EE0B695A795D9
:103E5000979587952A95D1F72681332744275527AB
:103E600082179307A407B50709F0E0C080E090E04F
:103E7000A0EEB0E0E822F9220A231B2375E1169593
:103E80000795F794E7947A95D1F72781822F9927A0
:103E9000AA27BB2787709070A070B070E816F9064B
:103EA0000A071B0709F0C2C0922E96949694969426
:103EB0008281A82FBB27838199279695982F8827E1
:103EC00097958795A82BB92B109709F4AFC0092DAA
:103ED000112700FF09C0C5014496AC0160E070E005
:103EE000CD010E943521DC01109729F0BD018091A0
:103EF0002F010E94EB1BD5018D919C91892B09F418
:103F000095C001FF93C0F5018685816086878EC0CC
:103F1000F6018281282F3327838199279695982F40
:103F2000882797958795282B392B30933703209333
:103F3000360352C0F6018281282F332783819927C7
:103F40009695982F882797958795282B392B30930E
:103F50003A032093390384818093470385818093BA
:103F60003B03868180933C038091380381601CC0B1
:103F7000F6013296ADE3B3E094E081918D939150D8
:103F800097FFFBCF8091380382600EC0D601129656
:103F9000EDE3F3E093E08D9185839150319697FFA7
:103FA000FACF8091380384608093380315C081E094
:103FB0008093B30111C00E94571CF60182810E94B8
:103FC000D80D0AC0F6018281882321F00E94741B5B
:103FD000FC0184810E94B10BD6018C9199278F77C7
:103FE000907020912F0133278217930749F4809115
:103FF0003503882329F08091350381508093350360
:10400000F50186859927969587959C0121703070DA
:1040100080FD04C0A90160E0C90106C0F50144812A
:1040200055816089808191810E94851CCE01019615
:104030000E94C306892B09F0C8CD2F960FB6F894BD
:10404000DEBF0FBECDBFDF91CF911F910F91FF90CB
:10405000EF90DF90CF90BF90AF909F900895CF9357
:10406000DF93CDB7DEB726970FB6F894DEBF0FBE4D
:10407000CDBF36E0FE01319611923A95E9F74983BA
:10408000AE014F5F5F4F0E94BB1D26960FB6F8949E
:10409000DEBF0FBECDBFDF91CF910895CF93DF93E9
:1040A000CDB7DEB726970FB6F894DEBF0FBECDBFF3
:1040B00026E0FE01319611922A95E9F7282F2F77F5
:1040C0002983880F892F881F990B91958F778A8371
:1040D000AE014F5F5F4F63E18FEF0E94BB1D2696DD
:1040E0000FB6F894DEBF0FBECDBFDF91CF9108951C
:1040F0009F92AF92BF92CF92DF92EF92FF920F9377
:104100001F93CF93DF93CDB7DEB726970FB6F89402
:10411000DEBF0FBECDBFFC018B01942E6901672B62
:1041200011F0232B19F480E090E085C086E05E0159
:104130000894A11CB11CD5011D928A95E9F754E1A0
:10414000E52E8E2F8F778983EE0FEF2FEE1FFF0B5B
:10415000F1958E2F8F778A8320E08E2D99278631D7
:10416000910501F18731910534F48431910549F0CD
:104170004597C9F024C08731910599F0489781F09F
:104180001EC0802F8F778B83C801880F892F881FCF
:10419000990B91958F778C83892D8F778D830FC0A5
:1041A00023E02D5F2D5F92E0D5011296F601E20F1C
:1041B000F11D80818D9391502F5F97FFF7CF109263
:1041C000370310923603FF24809136039091370312
:1041D000892B09F5AE014F5F5F4F6E2D8FEF0E9467
:1041E000BB1D85E08093350306C08091350388238D
:1041F00041F00E9471048091360390913703892B1E
:10420000A1F3F3948091360390913703892B19F42D
:1042100089E08F15F8F68091360390913703009767
:1042200051F0E0913603F0913703E39488E18E1565
:1042300008F087CFCF0126960FB6F894DEBF0FBEE9
:10424000CDBFDF91CF911F910F91FF90EF90DF9045
:10425000CF90BF90AF909F9008959A01462FBC01D8
:1042600080E090E00E9478200895DF92EF92FF9224
:104270000F931F93CF93DF93CDB7DEB726970FB67B
:10428000F894DEBF0FBECDBF9C017B018A01019770
:104290008F5F934008F050C086E0FE013196119286
:1042A0008A95E9F7822F8F778983220F232F221F88
:1042B000330B3195822F8F778A8310923803DD2458
:1042C00080913803873031F1AE014F5F5F4F60E17D
:1042D0008FEF0E94BB1D8FE08093350306C0809155
:1042E0003503882331F00E947104809138038730B0
:1042F000B1F780913803873029F082B799278896E3
:104300000E94DD08D39480913803873019F089E04A
:104310008D15D0F680913803873021F480913B03CE
:104320008F3769F4E114F10411F0F70110820115DF
:10433000110511F0F801108280E090E018C0E1143E
:10434000F10421F080914703F701808301151105E5
:1043500051F08BE0F801ABE3B3E00D9001928A9548
:10436000E1F7F80113868091390390913A0326967C
:104370000FB6F894DEBF0FBECDBFDF91CF911F9176
:104380000F91FF90EF90DF9008950F931F93CF93BD
:10439000DF93CDB7DEB726970FB6F894DEBF0FBE1A
:1043A000CDBF062F26E0FE01319611922A95E9F73E
:1043B000282F2F772983880F892F881F990B919594
:1043C0008F778A838FEF9FEF909337038093360325
:1043D00010E0809136039091370397FF20C0AE0123
:1043E0004F5F5F4F602F8FEF0E94BB1D85E0809372
:1043F000350306C080913503882341F00E94710483
:1044000080913603909137039923A4F31F5F809125
:1044100036039091370397FF02C01A3000F3809162
:1044200036039091370326960FB6F894DEBF0FBE81
:10443000CDBFDF91CF911F910F91089561E10E944F
:10444000C521089562E10E94C5210895E199FECF3A
:104450009FBB8EBBE09A99278DB3089541155105F6
:1044600069F0DC01E199FECF7FBB6EBBE09A6F5F24
:104470007F4F0DB20D9241505040B1F70895E19930
:10448000FECF9FBB8EBB6DBB0FB6F894E29AE19A4C
:104490000FBE0895DC0101C06D9341505040E0F71C
:1044A0000895FB01DC0101900D920020E1F70895D1
:1044B0000F931F93CF93DF93CDB7DEB72C970FB633
:1044C000F894DEBF0FBECDBF8C0136E03C838983FC
:1044D0009A832FEF3FE72D833E83CE0101960E9402
:1044E000AA22AF81B885A00FB11F1C922C960FB6DF
:1044F000F894DEBF0FBECDBFDF91CF911F910F911A
:1045000008950F931F93CF93DF93CDB7DEB72C970A
:104510000FB6F894DEBF0FBECDBF8C013EE03C83EA
:1045200089839A832FEF3FE72D833E83CE01019647
:104530000E94AA22AF81B885A00FB11F1C922C96B1
:104540000FB6F894DEBF0FBECDBFDF91CF911F91A4
:104550000F9108952F923F924F925F926F927F92A8
:104560008F929F92AF92BF92CF92DF92EF92FF9283
:104570000F931F93CF93DF93CDB7DEB762970FB63C
:10458000F894DEBF0FBECDBFAA24BB2465014C0149
:104590006D877E874F87588B44245524FC014682C3
:1045A0005782838181FD5BC28FEF9FEF6FC240FE18
:1045B00044C2862D80538A30E0F4F0E36F1641F454
:1045C0002A89222329F4772019F480E091E08BC016
:1045D0008AE09A89989F902D1124892F860D805307
:1045E0008A8B882314F4EFE7EA8B43FC38C27A887D
:1045F00036C243FE05C0FA89FF2311F421E02A8B5D
:10460000862D992787FD90958836910554F5853636
:1046100091050CF06BC08835910509F4D3C089353C
:104620009105B4F48B32910509F442C08C329105A6
:1046300044F48032910509F43FC0839709F442C0E5
:10464000F2C18D329105D9F18E9709F440C0EBC1CA
:104650008336910509F454C08436910509F478C075
:10466000E2C18037910509F4A5C08137910584F432
:104670008C369105B1F18D3691052CF48936910572
:1046800009F466C0D0C18F36910509F490C0CBC142
:104690008537910509F498C08637910524F483374E
:1046A0009105B9F1C0C18837910509F48BC0BBC130
:1046B00080E190E0482A592AE0E2F0E005C080E875
:1046C00090E011C0E0E4F0E04E2A5F2AC8C188E023
:1046D00090E0482A592AEFEFFEEF4E225F221A8A15
:1046E000BEC184E090E0482A592AB9C10F2EFFE3E9
:1046F000AF2EF02D7A940F2EF3E66F2EF02D3AC1E7
:10470000EF85F889CF0102968F87988BA0807A94E5
:1047100031C1EF85F889CF0102968F87988BA080F1
:10472000B18043FE0BC0EA898E2F992787FD9095B3
:10473000BC01C5010E949225898B07C0F50101903B
:104740000020E9F73197EA19E98BF9897F1A12C13C
:1047500042FE0BC0EF85F889CF0104968F87988BB6
:1047600020813181428153810DC0EF85F889CF01CD
:1047700002968F87988B808191819C01442737FD19
:104780004095542F59016A01552364F4E2E0F0E0AA
:104790004E2A5F2AD094C094B094A094A11CB11C5E
:1047A000C11CD11C8FEB9FEF482259222BC098E0EF
:1047B000998B0AC0E0E4F0E04E2A5F2A0F2EF8E75A
:1047C0006F2EF02DF0E1F98B42FE0BC0EF85F889DA
:1047D000CF0104968F87988B20813181428153814C
:1047E0000BC0EF85F889CF0102968F87988B808167
:1047F00091819C014427552759016A01EFECFFEF95
:104800004E225F221E010894211C311CF989EF2ED3
:10481000FF2400271127C601B501A80197010E94B6
:10482000A925DC01CB01F10180838A301CF0860DC3
:10483000815203C0F1018081805DF10181931F01EC
:10484000C601B501A80197010E94A92559016A0175
:104850002115310541055105F1F6CE010196A22C35
:10486000A81AC20182739070892B09F07A9446FECF
:104870000FC0872D992787FD9095F989F03131F484
:104880000F2EFEEF7F2EF02D780E02C0782E7A9438
:1048900043FE12C08A89282F332727FD30958A2DA1
:1048A0009927821793072CF0E7EFFFEF4E225F2244
:1048B00003C0FA89FA19FA8B43FE03C02A89721AD7
:1048C00001C07A18C20180789170892B69F4872D14
:1048D0007A9418164CF4B40180E290E00E945F25AF
:1048E000872D7A941816BCF341FE04C0B4018DE202
:1048F00090E00BC044FE04C0B4018BE290E005C020
:1049000045FE05C0B40180E290E00E945F2546FEAE
:104910000FC0B40180E390E00E945F258989803157
:1049200039F4862D992787FD9095B4010E945F2563
:1049300050FE0DC0872D7A9418164CF4B40180E314
:1049400090E00E945F25872D7A941816BCF343FEF1
:1049500011C08A89982F91509A8B18165CF4B40173
:1049600080E390E00E945F258A89E82FE150EA8B7E
:104970001816ACF3842D807869F4872D7A94181674
:104980004CF4B40180E290E00E945F25872D7A9478
:104990001816BCF3F3E66F1641F48A2D992787FDAC
:1049A0009095B4010E945F252DC023E76216B1F4F3
:1049B00089898150898B8F3F29F1F5018081992761
:1049C00087FD90950894A11CB11CB4010E945F253D
:1049D00099899150998B9F3F81F714C0CE01019620
:1049E0002816390679F08E010F5F1F4FF101829171
:1049F0001F01992787FD9095B4010E945F2520161D
:104A00003106A1F7842D8078A9F0872D7A941816A5
:104A10008CF4B40180E290E00E945F25872D7A94A7
:104A20001816BCF307C0862D992787FD9095B40111
:104A30000E945F254424552412C0F5E26F1641F40C
:104A40004424552443941A8A7A882AE0298B07C083
:104A5000862D992787FD9095B4010E945F25F4016A
:104A6000838183FF08C0ED85FE85CF0101968D8788
:104A70009E87649005C0ED85FE856190ED87FE8779
:104A8000662009F094CDF4018681978162960FB675
:104A9000F894DEBF0FBECDBFDF91CF911F910F9174
:104AA000FF90EF90DF90CF90BF90AF909F908F904E
:104AB0007F906F905F904F903F902F9008950F934D
:104AC0001F93CF93DF938C01EB018B81992781FF9B
:104AD00022C082FF14C02E813F814C815D8124174A
:104AE00035073CF4A881B9810D93A883B9832E8141
:104AF0003F812F5F3F4F2E833F83C8010EC0E88563
:104B0000F985802F0995892B31F4EE81FF8131964B
:104B1000EE83FF83F2CF8FEF9FEFDF91CF911F9155
:104B20000F910895FC016150704001900110D8F779
:104B3000809590958E0F9F1F0895991B79E004C072
:104B4000991F961708F0961B881F7A95C9F78095CC
:104B50000895A1E21A2EAA1BBB1BFD010DC0AA1FBE
:104B6000BB1FEE1FFF1FA217B307E407F50720F0D6
:104B7000A21BB30BE40BF50B661F771F881F991F51
:104B80001A9469F760957095809590959B01AC019A
:064B9000BD01CF010895F4
:104B9600FFFF00010000FF0000D616FF000074169C
:104BA600FF0000D412FF00001A13FF01002615FFB4
:104BB60001002C13FF01004F14FF01002316FFFF15
:00000001FF
